:10000000F0288030A100FE30A4200130A4207530FB
:10001000A6003030BB28A101A117AE00FE30A420FD
:100020002E08A428A401A900AA01A01124080319DC
:10003000A0151030A3000301A90DAA0D031801306B
:1000400045202308031D1B280800A401A900AA01BC
:10005000A01124080319A0150530A3002730A8001B
:1000600010303E200330A800E8303E20A801643064
:100070003E20A8010A303E2029084528A7002A086A
:10008000A6002908A500CF202508A500A303031971
:10009000A011240803194F28230203185628250805
:1000A000031DA011A0195628303EA4280800AC005A
:1000B000061186118316061186110F3086058312EC
:1000C0002C08A01881283E30A6008030BB20333099
:1000D000AB0095201330A6008830BB2095206430FB
:1000E000BA2095206430BA202230AB009520283009
:1000F00080200C30802006308020A0142C0881281D
:100100002014AB00201C8F288611033C031C94286C
:1001100094200530A600DC30BB2003140800201416
:10012000FE3C0319A2288615201C201006150F304E
:1001300086052B08F03986040611AB0E2018952889
:100140003230BA202C08EB28A11B572883178001D6
:10015000840AFF3E031DA728EB28A801A700FF3053
:10016000A707031CA807031CEB280330A600DF30F9
:10017000BB20AF28A601E83EA500A609FC30031C61
:10018000C428A5070318C128A5070000A60FC12889
:100190002518CA28A51CCE280000CE280800AA01D0
:1001A000A9011030AB00260DA90DAA0D2708A90240
:1001B0002808031C280FAA020318E5282708A90706
:1001C00028080318280FAA070310A50DA60DAB0BCE
:1001D000D3282508EB28831383120313000008009B
:1001E000A00107309F00F03083168500FF308600A5
:1001F000811320308400603083128A01A720A03050
:10020000840050308A01A7202030840050308A01B9
:10021000A6200130A800F4308A01AE208A01012016
:1002200052308A01572043308A01572035308A01E5
:10023000572020308A0157204E308A0157206130E4
:100240008A0157206D308A01572065308A01572076
:100250006E308A01572020308A0157204E308A01A3
:1002600057204C308A01572020308A0157205630C1
:100270008A0157202D308A01572031308A015720BA
:100280008A116A29051A3115051E3111B6010301BB
:10029000051A013E3119013C03190130031D030108
:1002A000B0003230360201300318030130058A11E4
:1002B00003195D29B60A8A014729323036028A11AC
:1002C000031D64298A15E12F0430A6004C308A01F1
:1002D000BB20080005110510851006183114061CF6
:1002E0003110B6018A11051E77298A017229013061
:1002F000051A0301B000343036020130031803013F
:1003000030058A1103198729B60A8A017729343002
:1003100036028A1103188E298A15D92F3208B300A4
:100320003408B50005150130A600F4308A01BB2061
:100330008A014221030131190130013A03193213B4
:10034000031D32178A014221B114311DB1108A01F7
:1003500042213416311D34128A014221B415311D57
:10036000B4118A0142213415311D34118A01422110
:10037000B414311DB4108A0142213414311D3410DB
:100380008A014221B216311DB2128A01422132166F
:10039000311D32128A014221B215311DB2118A017A
:1003A00042213215311D32118A014221B214311D10
:1003B000B2108A0142213214311D32103408350244
:1003C000031D0130B00032083302031D0130300438
:1003D000B000060831060139031D013030048A15CA
:1003E0000319D42F8A0101208A15061C9F2F340877
:1003F0008A11031D032A54308A01572056308A017E
:1004000057208A11712C013034028A11031D132ADE
:1004100054308A01572056308A01572032308A01E1
:1004200057208A11712C023034028A11031D322A9E
:1004300054308A01572065308A0157206C308A0178
:10044000572065308A01572074308A015720653063
:100450008A01572078308A01572074308A0157204A
:100460008A11712C033034028A11031D512A56302F
:100470008A01572069308A01572064308A01572049
:1004800065308A0157206F308A01572020308A0159
:10049000572056308A01572044308A0157208A114C
:1004A000712C043034028A11031D732A56308A01DC
:1004B000572069308A01572064308A0157206530FF
:1004C0008A0157206F308A01572020308A01572037
:1004D0004C308A01572056308A01572031308A012A
:1004E00057208A11712C053034028A11031D862A87
:1004F00056308A01572043308A01572052308A01F2
:10050000572031308A0157208A11712C063034026D
:100510008A11031D992A56308A01572043308A01D7
:10052000572052308A01572032308A0157208A11D1
:10053000712C083034028A11031DA92A53308A0114
:10054000572041308A01572054308A0157208A11A0
:10055000712C093034028A11031DC22A43308A01EA
:10056000572061308A0157206D308A01572065304D
:100570008A01572072308A01572061308A01572042
:100580008A11712C0A3034028A11031DD52A533086
:100590008A01572041308A01572054308A01572060
:1005A00032308A0157208A11712C0C3034028A11A2
:1005B000031DE52A43308A01572044308A01572021
:1005C00056308A0157208A11712C0D3034028A115D
:1005D000031D072B43308A01572061308A015720C1
:1005E0006D308A01572063308A0157206F308A01AD
:1005F000572072308A01572064308A0157206530B5
:100600008A01572072308A0157208A11712C1030CC
:1006100034028A11031D2C2B56308A015720653075
:100620008A01572072308A01572073308A0157207F
:1006300074308A01572065308A01572072308A0150
:1006400057206B308A01572065308A01572072305D
:100650008A0157208A11712C113034028A11031D2E
:10066000422B54308A01572075308A0157206E3052
:100670008A01572065308A01572072308A0157203D
:100680008A11712C123034028A11031D552B5430FB
:100690008A01572061308A01572070308A01572023
:1006A00065308A0157208A11712C133034028A1167
:1006B000031D852B56308A0157206F308A01572041
:1006C0008A01572072308A01572076308A015720DC
:1006D00065308A01572072308A01572073308A01B1
:1006E000572074308A01572065308A0157207230B4
:1006F0008A0157206B308A01572065308A015720C4
:1007000072308A0157208A11712C143034028A11F8
:10071000031D922B43308A01572044308A01572011
:100720008A11712C153034028A11031DAE2B503002
:100730008A01572069308A01572063308A01572087
:100740006B308A0157202D308A01572075308A017D
:10075000572070308A0157208A11712C17303402CB
:100760008A11031DDC2B44308A01572069308A012D
:10077000572067308A01572069308A01572074302A
:100780008A01572061308A0157206C308A01572036
:1007900065308A01572020308A01572074308A0141
:1007A000572061308A01572070308A015720653008
:1007B0008A0157208A11712C1A3034028A11031DC4
:1007C000EC2B43308A01572044308A0157205230A5
:1007D0008A0157208A11712C1D3034028A11031DA1
:1007E000142C56308A01572065308A015720723008
:1007F0008A0157206C308A01572069308A015720BE
:1008000063308A01572068308A01572074308A018A
:10081000572069308A0157206E308A01572067308F
:100820008A0157208A11712C1E3034028A11031D4F
:10083000422C56308A01572065308A015720723089
:100840008A0157206C308A01572069308A0157206D
:1008500063308A01572068308A01572074308A013A
:10086000572069308A0157206E308A01572067303F
:100870008A01572020308A01572032308A015720C0
:100880008A11712C1F3034028A11031D602C5430E0
:100890008A01572065308A0157206C308A01572021
:1008A00065308A01572066308A0157206F308A01EF
:1008B00057208A0157206E308A0157208A11712CE7
:1008C00053308A01572079308A01572073308A01CA
:1008D00057203A308A0157208030A10034088A011D
:1008E0002520C0308A010B20A1010A3032028A1172
:1008F0000318932C54308A0157206F308A015720F7
:1009000065308A01572074308A01572073308A017C
:10091000572020308A0157208030A10032088A01F8
:1009200025208A159D2F0A3032028A11031DA52C1D
:100930002D308A0157202F308A0157202D308A010F
:1009400057208A0157208A159D2F0B3032028A11B9
:10095000031D012D34088A11031DB92C43308A016F
:1009600057202F308A01572050308A0157208A1192
:10097000FF2C053034028A110319E72C06303402AB
:100980008A11031DE92C43308A0157202F308A0138
:10099000572050308A01572020308A0157202F30AD
:1009A0008A01572020308A01572053308A0157206E
:1009B00065308A0157206C308A01572065308A01E2
:1009C000572063308A01572074308A0157208A11DA
:1009D000FF2C143034028A110319FF2C1730340213
:1009E0008A11031DFF2C54308A01572069308A0177
:1009F00057206D308A01572065308A0157208A15AB
:100A00009D2F0C3032028A11031D202D53308A0194
:100A1000572074308A01572061308A0157206E3088
:100A20008A01572064308A0157202D308A015720CF
:100A300062308A01572079308A0157208A159D2F0C
:100A40000D3032028A11031D332D4D308A0157209B
:100A500075308A01572074308A01572065308A0129
:100A600057208A159D2F0E3032028A11031D792DD1
:100A700034088A11031D552D56308A0157206F30D6
:100A80008A0157208A01572072308A0157206B3023
:100A90008A01572065308A01572075308A01572016
:100AA00072308A0157208A11772D053034028A115D
:100AB0000319772D063034028A11031D772D543027
:100AC0008A01572072308A01572061308A015720ED
:100AD00063308A0157206B308A01572069308A01C0
:100AE00057206E308A01572067308A0157208A15B7
:100AF0009D2F0F3032028A11031D8C2D49308A013F
:100B000057206E308A01572066308A0157206F3097
:100B10008A0157208A159D2F103032028A11031D39
:100B2000AB2D56308A0157206F308A0157206C3028
:100B30008A01572075308A0157206D308A0157206D
:100B400065308A01572020308A0157202B308A01D6
:100B500057208A159D2F113032028A11031DCA2D8C
:100B600056308A0157206F308A0157206C308A0135
:100B7000572075308A0157206D308A015720653023
:100B80008A01572020308A0157202D308A015720B2
:100B90008A159D2F123032028A11031DF52D48301F
:100BA0008A01572065308A0157206C308A0157200E
:100BB00064308A01572065308A01572072308A01DB
:100BC000572068308A01572065308A0157206930E4
:100BD0008A01572064308A01572020308A0157202B
:100BE0002B308A0157208A159D2F133032028A112B
:100BF000031D202E48308A01572065308A01572076
:100C00006C308A01572064308A01572065308A0190
:100C1000572072308A01572068308A01572065308A
:100C20008A01572069308A01572064308A01572091
:100C300020308A0157202D308A0157208A159D2F98
:100C4000143032028A11031D3C2E4B308A0157208A
:100C50006C308A01572065308A01572075308A012F
:100C6000572072308A01572020308A0157202B30BC
:100C70008A0157208A159D2F153032028A11031DD3
:100C8000582E4B308A0157206C308A01572065302E
:100C90008A01572075308A01572072308A01572007
:100CA00020308A0157202D308A0157208A159D2F28
:100CB000163032028A11031D702E42308A015720ED
:100CC00061308A01572073308A0157208A015720EA
:100CD00020308A0157202B308A0157208A159D2FFA
:100CE000173032028A11031D882E42308A015720A4
:100CF00061308A01572073308A0157208A015720BA
:100D000020308A0157202D308A0157208A159D2FC7
:100D1000183032028A11031DA72E54308A01572041
:100D200072308A01572065308A01572062308A016B
:100D300057206C308A01572065308A0157202030B7
:100D40008A0157202B308A0157208A159D2F193090
:100D500032028A11031DC62E54308A015720723088
:100D60008A01572065308A01572062308A01572056
:100D70006C308A01572065308A01572020308A0163
:100D800057202D308A0157208A159D2F1A303202A4
:100D90008A11031DE52E42308A01572061308A01F5
:100DA00057206C308A01572061308A0157206E30FD
:100DB0008A01572073308A01572020308A0157203A
:100DC00052308A0157208A159D2F1B3032028A111A
:100DD000031D042F42308A01572061308A015720B9
:100DE0006C308A01572061308A0157206E308A01A9
:100DF000572073308A01572020308A0157204C3009
:100E00008A0157208A159D2F1C3032028A11031D3A
:100E10003D2F143034028A11031D242F53308A01D0
:100E2000572068308A01572075308A015720663074
:100E30008A0157208A0157206C308A01572065307B
:100E40008A0157208A113B2F173034028A11031D63
:100E50003B2F52308A01572065308A01572070306D
:100E60008A01572065308A01572061308A01572056
:100E700074308A0157208A159D2F1D3032028A1145
:100E8000031D762F053034028A1103195B2F0630BB
:100E900034028A11031D5D2F54308A0157206930B6
:100EA0008A0157206D308A01572065308A0157200A
:100EB00072308A0157208A11742F143034028A113B
:100EC000031D742F52308A01572065308A01572044
:100ED00070308A01572065308A01572061308A01BD
:100EE000572074308A0157208A159D2F1E303202F8
:100EF0008A11031DC72F053034028A110319A62F4A
:100F0000063034028A11031DA82F52308A0157205F
:100F100065308A01572063308A0157206F308A017B
:100F2000572072308A01572064308A0157202030C0
:100F30008A0157206D308A0157206F308A0157206F
:100F400064308A01572065308A0157208A11C52FE5
:100F5000113034028A11031DC52F53308A015720E6
:100F600065308A01572061308A01572072308A012A
:100F7000572063308A01572068308A01572020307B
:100F80008A0157202B308A0157208A159D2F1F3048
:100F900032028A15031D2128053034028A150319EF
:100FA0000028063034028A15031D022846308A01C3
:100FB000572061308A01572073308A0157207430DE
:100FC0008A01572020308A01572072308A01572029
:100FD00065308A01572076308A01572065308A01B2
:100FE000572072308A01572073308A0157206530AC
:100FF0008A01572020308A01572031308A0157203A
:101000008A151F28113034028A15031D1F285330FA
:101010008A01572065308A01572061308A015720A4
:1010200072308A01572063308A01572068308A0164
:10103000572020308A0157202D308A0157208A15E9
:101040009D2F203032028A15031D482850308A0116
:10105000572072308A0157206F308A01572067303D
:101060008A01572072308A01572061308A01572047
:101070006D308A0157208A01572061308A0157203C
:1010800020308A0157202B308A0157208A159D2F46
:10109000213032028A15031D6F2850308A015720F3
:1010A00072308A0157206F308A01572067308A01D9
:1010B000572072308A01572061308A0157206D30E5
:1010C0008A0157208A01572061308A015720203039
:1010D0008A0157202D308A0157208A159D2F2230F2
:1010E00032028A15031DCF2834088A15031D832870
:1010F00050308A0157203C308A01572050308A01F5
:1011000057208A15CD28053034028A150319B128D5
:10111000063034028A15031DB32853308A01572044
:101120006C308A0157206F308A01572077308A014E
:10113000572020308A01572072308A0157206530AD
:101140008A01572076308A01572065308A0157205E
:1011500072308A01572073308A01572065308A0126
:1011600057208A15CD28143034028A15031DCD2846
:1011700049308A0157206E308A01572064308A0135
:10118000572065308A01572078308A015720203057
:101190008A0157202B308A0157208A159D2F233032
:1011A00032028A15031D3E2934088A15031DE528DD
:1011B00049308A0157202F308A01572049308A014F
:1011C00057208A0157208A153C29053034028A1598
:1011D00003190D29063034028A15031D0F294130E9
:1011E0008A01572075308A01572064308A015720C0
:1011F00069308A0157206F308A01572020308A01D8
:1012000057206D308A0157206F308A015720643093
:101210008A01572065308A0157208A153C291030F1
:1012200034028A15031D22294C308A01572053307D
:101230008A0157202D308A01572041308A015720DA
:101240008A153C29143034028A15031D3C29493083
:101250008A0157206E308A01572064308A01572056
:1012600065308A01572078308A01572020308A0162
:1012700057202D308A0157208A159D2F25303202A4
:101280008A15031D662953308A01572074308A015C
:10129000572065308A01572072308A015720653007
:1012A0008A0157206F308A0157202F308A0157203A
:1012B0004D308A0157206F308A0157206E308A01E5
:1012C00057206F308A0157208A159D2F2730320210
:1012D0008A15031D9329053034028A1503197E29C6
:1012E000063034028A15031D80294F308A015720A9
:1012F00054308A01572052308A0157208A1591298B
:10130000103034028A15031D91294C308A01572070
:1013100053308A0157202D308A01572042308A01EC
:1013200057208A159D2F283032028A15031DBE29A9
:1013300053308A0157206C308A0157206F308A0160
:10134000572077308A01572020308A0157204630B5
:101350008A0157206F308A01572072308A01572046
:1013600077308A01572061308A01572072308A0114
:10137000572064308A0157208A159D2F2930320268
:101380008A15031D142A34088A15031DDD295430DB
:101390008A0157208A01572020308A01572048307F
:1013A0008A0157206F308A0157206C308A015720FC
:1013B00064308A0157208A15122A053034028A15B2
:1013C0000319F629063034028A15031DF829503016
:1013D0008A01572061308A01572075308A015720D1
:1013E0007A308A01572065308A0157208A15122ADF
:1013F000143034028A15031D122A50308A015720F6
:1014000072308A0157206F308A01572067308A0175
:10141000572072308A01572061308A0157206D3081
:101420008A0157208A159D2F2A3032028A15031D02
:10143000912A34088A15031D332A54308A01572013
:101440008A01572020308A01572054308A015720C2
:1014500069308A0157206A308A01572064308A0136
:1014600057208A158F2A053034028A150319672AF6
:10147000063034028A15031D692A46308A01572036
:1014800061308A01572073308A01572074308A01F5
:10149000572020308A01572046308A0157206F306C
:1014A0008A01572072308A01572077308A015720ED
:1014B00061308A01572072308A01572064308A01D6
:1014C000572020308A01572031308A0157208A1551
:1014D0008F2A173034028A15031D8F2A52308A0151
:1014E000572065308A01572063308A0157206F30BA
:1014F0008A01572072308A01572064308A015720B0
:1015000020308A0157206D308A01572075308A01BA
:10151000572074308A01572065308A0157208A1578
:101520009D2F2B3032028A15031DCD2A34088A15CF
:10153000031DBF2A54308A0157208A0157202030CA
:101540008A01572056308A01572065308A0157207A
:1015500072308A01572067308A01572072308A0121
:1015600057206F308A01572074308A015720653028
:101570008A0157206E308A0157208A15CB2A5330B2
:101580008A01572063308A01572061308A01572031
:101590006E308A0157208A159D2F2C3032028A1511
:1015A000031D322B34088A15031DE32A54308A01A7
:1015B00057208A01572020308A0157203F308A0166
:1015C00057208A15302B053034028A150319172B42
:1015D000063034028A15031D192B46308A01572024
:1015E00061308A01572073308A01572074308A0194
:1015F000572020308A01572072308A0157206530E9
:101600008A01572076308A01572065308A01572099
:1016100072308A01572073308A01572065308A0161
:10162000572020308A01572032308A0157208A15EE
:10163000302B123034028A15031D302B44308A01BE
:10164000572065308A01572063308A0157206B305C
:101650008A01572020308A01572041308A015720C3
:101660008A159D2F2D3032028A15031D622B3408F6
:101670008A15031D512B54308A0157208A015720A7
:1016800020308A0157204D308A01572075308A0159
:10169000572074308A01572065308A0157208A15F7
:1016A000602B45308A0157206A308A015720653007
:1016B0008A01572063308A01572074308A015720ED
:1016C0008A159D2F2E3032028A15031DCD2B34082A
:1016D0008A15031D7E2B54308A0157208A0157201A
:1016E00020308A0157204D308A01572069308A0105
:1016F000572078308A0157208A15CB2B05303402C9
:101700008A150319B22B063034028A15031DB42B37
:1017100046308A01572061308A01572073308A0190
:10172000572074308A01572020308A0157204630D4
:101730008A0157206F308A01572072308A01572062
:1017400077308A01572061308A01572072308A0130
:10175000572064308A01572020308A0157203230C8
:101760008A0157208A15CB2B123034028A15031DAB
:10177000CB2B44308A01572065308A0157206330D3
:101780008A0157206B308A01572020308A01572068
:1017900042308A0157208A159D2F2F3032028A1538
:1017A000031DFC2B143034028A15031DE52B463033
:1017B0008A01572061308A01572073308A015720EF
:1017C00074308A0157208A15FA2B52308A0157202B
:1017D00065308A01572076308A01572065308A01AA
:1017E000572072308A01572073308A0157206530A4
:1017F0008A0157208A159D2F303032028A15031D29
:10180000122C50308A01572061308A0157207530E0
:101810008A0157207A308A01572065308A01572083
:101820008A159D2F313032028A15031D282C523023
:101830008A01572065308A01572073308A0157206A
:1018400065308A01572074308A0157208A159D2FF0
:10185000323032028A15031D412C52308A01572042
:1018600065308A01572077308A01572069308A0114
:1018700057206E308A01572064308A0157208A151C
:101880009D2F333032028A15031D542C47308A01B4
:1018900057206F308A01572054308A0157206F300B
:1018A0008A0157208A159D2F343032028A15031D74
:1018B000672C57308A01572069308A0157206E30D3
:1018C0008A01572064308A0157208A159D2F3530B0
:1018D00032028A15031D7A2C50308A0157206C3051
:1018E0008A01572061308A01572079308A015720B8
:1018F0008A159D2F363032028A15031D8D2C5330E8
:101900008A01572074308A0157206F308A0157208E
:1019100070308A0157208A159D2F373032028A1580
:10192000031DA62C4F308A01572070308A015720A2
:101930006E308A01572061308A0157206D308A014C
:10194000572065308A0157208A159D2F3830320282
:101950008A15031DBF2C45308A01572078308A0133
:10196000572074308A01572065308A015720723021
:101970008A0157206E308A0157208A159D2F3A30F0
:1019800032028A15031DD52C53308A01572050305E
:101990008A0157202F308A0157204C308A01572066
:1019A00050308A0157208A159D2F3C3032028A150B
:1019B000031DF42C54308A01572065308A015720CA
:1019C0006C308A01572065308A01572074308A01B3
:1019D000572065308A01572078308A0157207430AB
:1019E0008A0157208A159D2F3F3032028A15031D28
:1019F0000C2D54308A01572056308A015720203050
:101A00008A01572061308A0157208A0157206E30A1
:101A10008A0157208A159D2F4F3032028A15031DE7
:101A20001F2D56308A01572069308A0157206530B2
:101A30008A01572077308A0157208A159D2F503010
:101A400032028A15031D372D4F308A0157206D3021
:101A50008A01572068308A0157206F308A01572049
:101A60008A01572067308A0157208A159D2F5130EF
:101A700032028A15031D4F2D4F308A0157206D30D9
:101A80008A0157206C308A01572061308A01572023
:101A90008A01572067308A0157208A159D2F5230BE
:101AA00032028A15031D622D4D308A0157206530A0
:101AB0008A0157206E308A01572075308A015720DD
:101AC0008A159D2F553032028A15031D782D4C3012
:101AD0008A01572069308A0157206E308A015720C9
:101AE0006B308A01572073308A0157208A159D2F49
:101AF000563032028A15031D912D52308A0157202B
:101B000065308A01572063308A01572068308A0186
:101B1000572074308A01572073308A0157208A1564
:101B20009D2F573032028A15031D9E2D4F308A019A
:101B300057204B308A0157208A159D2F5D30320285
:101B40008A15031DB62D46308A01572072308A014E
:101B5000572065308A0157208A0157207A308A0140
:101B6000572065308A0157208A159D2F6130320237
:101B70008A15031DC62D44308A0157204E308A0134
:101B8000572052308A0157208A159D2F6B30320220
:101B90008A15031DD82D52308A0157206F308A01D3
:101BA00057208A01572064308A0157208A159D2FBB
:101BB0006C3032028A15031D022E34088A15031D6B
:101BC000F22D47308A01572072308A0157206F303A
:101BD0008A01572065308A0157206E308A015720CC
:101BE0008A15002E143034028A15031D002E46304B
:101BF0008A01572054308A01572053308A015720D8
:101C00008A159D2F6D3032028A15031D142E473020
:101C10008A01572065308A0157208A0157206C308D
:101C20008A0157208A159D2F6E3032028A15031DB6
:101C30002A2E42308A0157206C308A0157206130A9
:101C40008A01572075308A01572077308A01572042
:101C50008A159D2F6F3032028A15031D3A2E573098
:101C60008A01572069308A01572074308A01572031
:101C70008A159D2F703032028A15031D562E493069
:101C80008A0157206E308A01572064308A0157201C
:101C900065308A01572078308A01572020308A0128
:101CA00057202B308A0157208A159D2F7130320220
:101CB0008A15031D722E49308A0157206E308A0121
:101CC000572064308A01572065308A0157207830C8
:101CD0008A01572020308A0157202D308A01572051
:101CE0008A159D2F723032028A15031D9D2E5330A6
:101CF0008A01572074308A01572061308A015720A9
:101D000072308A01572074308A01572020308A01AE
:101D100057206D308A01572061308A015720723078
:101D20008A0157206B308A01572065308A0157207D
:101D300072308A0157208A159D2F753032028A151C
:101D4000031DDE2E34088A15031DC62E4F308A016E
:101D500057206E308A01572064308A015720653041
:101D60008A01572072308A01572074308A01572027
:101D700069308A01572074308A01572065308A0102
:101D800057206C308A0157208A15DC2E1730340218
:101D90008A15031DDC2E41308A01572070308A01DC
:101DA00057208A01572065308A0157206E308A01FA
:101DB000572064308A0157208A159D2F78303202CF
:101DC0008A15031DF42E46308A01572061308A019E
:101DD000572064308A01572065308A0157207230BD
:101DE0008A0157208A159D2F7A3032028A15031DE9
:101DF000422F053034028A150319322F063034027F
:101E00008A15031D342F54308A01572065308A010A
:101E100057206C308A0157208A01572065308A018B
:101E2000572072308A01572020308A0157202F30E6
:101E30008A01572020308A0157204D308A015720CF
:101E40006F308A0157206E308A01572069308A012D
:101E5000572074308A0157206F308A015720723022
:101E60008A0157208A15402F54308A015720653047
:101E70008A01572078308A01572074308A01572010
:101E80008A159D2F7E3032028A15031D8C2F34084F
:101E90008A15031D6F2F42308A01572065308A0151
:101EA00057208A0157206C308A01572064308A01FC
:101EB000572066308A0157206F308A0157207230D0
:101EC0008A0157206D308A01572061308A015720DE
:101ED0008A01572074308A0157208A158A2F0530CD
:101EE00034028A1503198A2F063034028A15031D1D
:101EF0008A2F54308A01572065308A0157206C3070
:101F00008A0157208A01572065308A015720723094
:101F10008A0157208A159D2F43308A0157206F3040
:101F20008A0157206D308A0157203A308A015720A4
:101F30008030A10032088A0125208A15D42F533021
:101F40008A01572079308A01572073308A0157203F
:101F50003A308A0157208030A10034088A012520B8
:101F60008030A10088308A010B2034088A011220B9
:101F70008030A100C0308A010B2043308A015720F5
:101F80006F308A0157206D308A0157203A308A011C
:101F9000572032088A0125208030A100C8308A01EC
:101FA0000B2032088A0112208515B11C85118A0187
:101FB0006A2905140130A800F4308A01AE208A0194
:101FC0006A29051185140130A800F4308A01AE2079
:0C1FD0003308B2003508B4008A016A2909
:02400E00303F41
:00000001FF
